:020000000528D1
:10000800082E8B13831203138312031385018601B1
:100018008316FF30831603138500FF308600831292
:100028008B138730831681008312C330A600A70183
:10003800831203138100A0308B0083160313A801D9
:10004800FF30AB01AC01AD00AE00952B8316031356
:10005800AA000310280DAB3E8400831329088000F2
:10006800840A2A088000A80A2808013A0319A80166
:100078000310280D8313AB3E84000008840A000493
:1000880003193728801B372800088A0084030008D2
:10009800820004307302031C5528031D55280030C4
:1000A8007202031858286728013083160313AA0020
:1000B8000030A9000000A90B5E2800000030F20201
:1000C800031CF3034D2800307302031C6F28031D23
:1000D8006F28043072020318722882287308831666
:1000E8000313AA007208A9000310AA0CA90C031094
:1000F800AA0CA90C0000A90B7E2800000800831296
:10010800031367086804031D8A289A2883160313B3
:10011800AA01FA30A9000000A90B8F2800000130BD
:1001280083120313E702031CE803832808008312E1
:100138000313851508008312031385110800831221
:1001480003130515720EF03986040F38860505115C
:1001580008009F20831203136708F200F20E0F3085
:10016800F205A320831203136708F200A320F3010A
:100178002830F2004D2008009B20831203136708E3
:10018800F200F20E0F30F205A32083120313670862
:10019800F200A320F3013230F2004D20080083164C
:1001A800031306128612061386138511051183128E
:1001B8000313E8010F30E70083209F200330F2008B
:1001C800A32083120313E8010530E70083200330DE
:1001D800F200A320F3016430F2004D200330F20056
:1001E800A32083120313E8010530E70083200230BF
:1001F800F200A320F3012830F2004D2028308312AA
:100208000313E700AD20083083120313E700AD2085
:100218000F3083120313E700AD200130831203135C
:10022800E700AD2083120313E8010230E7008320C2
:10023800063083120313E700AD20831203135C0812
:100248008A005B088200831203135E080139E70005
:10025800E70EE70DE70DC030E7058030E7045D08DD
:100268003F39E704AD20831203135C088A005B085A
:100278008200013083120313DC004730DB000030BA
:100288008A00D33082008312031352088A0051086F
:100298008200831203135308DD005408DE00013086
:1002A800DC005B30DB0001308A00273082008312DB
:1002B800031352088A0051088200831203135D0851
:1002C800E700C020831203135C088A005B088200E1
:1002D80073298312031354088A00530882006D217E
:1002E80083120313D5005508003A031D7C29992968
:1002F800831203135508DD000130DC008830DB0071
:1003080001308A006130820083120313D30A031973
:10031800D40A94298312031354088A0053088200CC
:100328008E2183120313D5007729831203135208F1
:100338008A0051088200831203135408D700530817
:10034800023E0318D70A83135718831784005508E9
:1003580080008313541883175308840080015408BD
:10036800D7005308013E0318D70A83135718831779
:100378008400800152088A00510882008312031306
:100388006008E4005F08013E0318E40A8313641858
:10039800831784000008E1008313601883175F083F
:1003A8008400000861060319DA29E529831203137A
:1003B800DC010130FF3ADC09013E0319DC0ADB00ED
:1003C8001C2A83120313E401033061070318E40AAB
:1003D8005F07E3000318E40A6008E407831364185E
:1003E8008317630884000008E200E10A6008E4005B
:1003F8005F08023E0318E40A831364188317840015
:10040800000861020318092A0C2A83120313E10168
:100418006008E4005F08013E0318E40A83136418C7
:100428008317840061088000DC016208DB001C2A55
:10043800831203135E088A005D0882008313831207
:1004480003136B1883176A0884000008013EED0047
:100458006B08EF006A08023E0318EF0A83136F184F
:100468008317840000086D0203183B2A3E2A831272
:100478000313ED016B08EF006A08013E0318EF0A49
:1004880083136F188317840000086D0603194D2A1B
:10049800542A013083120313E700E709E70A762A92
:1004A8008313831203136B1883176A088400EF0100
:1004B8000008033E0318EF0A6A07EE000318EF0A64
:1004C8006B08EF0783136F1883176E0884006C0896
:1004D800800083136B1883176A0884006D088000F6
:1004E800E701762A8312031369088A0068088200E4
:1004F800831603130C12831203135C088A005B082B
:100508008200831603130C1640308B0483120313E6
:1005180068088A0067088200831603138C12831206
:1005280003135C088A005B088200831603138C1689
:1005380040308B048312031352088A00510882004A
:10054800831603139816831203135C088A005B084A
:1005580082008312031318165C088A005B08820065
:100568008316031318080239003A03090439031DD6
:10057800013083120313E700C12A831203136908A9
:100588008A00680882001930831603139900181529
:1005980018128312031398170230DC00D830DB00DE
:1005A80002308A007C308200023083120313DC00A0
:1005B800E230DB0002308A00903082000630831679
:1005C8000313860418138312031318130230DC0074
:1005D800F230DB0002308A00A4308200023083123D
:1005E8000313DC00FC30DB0002308A00AD308200EF
:1005F8008312031352088A005108820083120313DE
:10060800EB013330EA005E08EC000330E9001130FA
:10061800E80002308A002230820083120313670840
:10062800DF000330E9001D30E80002308A00B430F2
:10063800820083120313E7080319232B242B2E2B84
:10064800033083120313E8002E30E70002308A00DB
:1006580085308200831203135F08DB00332B83127B
:1006680003135D088A005C08820083120313E0010B
:100678002030DF000330DE004630DD0001308A0024
:10068800C2308200831203135C08D2005B08D100D9
:100698004D2B8312031354088A00530882005A2BE7
:1006A8008312031354088A005308820054238312C8
:1006B8000313D5005508003A031D632B8F2B031134
:1006C8000319672B682B7E2B831203135508DE0052
:1006D8000330DD007430DC0003308A000230820011
:1006E800831203135B08D600D60803197C2B7D2BD5
:1006F8007E2B632B83120313D30A0319D40A8A2B84
:100708008312031354088A00530882008423831237
:100718000313D5005E2B8312031352088A00510875
:1007280082000730831203139F00831603130510FA
:1007380083120313D4012030D3001030D5000330C6
:10074800D200AB30D10001308A009F308200831282
:100758000313D4013330D3001030D5000330D20056
:10076800BA30D10001308A009F30820003308312F2
:100778000313D200C430D10002308A00C73082008F
:10078800033083120313D200CE30D10001308A0027
:100798003D308200033083120313E800D830E700AD
:1007A80002308A0085308200033083120313D2009E
:1007B800E230D10002308A009930820040308B0448
:1007C800413083120313CC00D301D4010330D2008B
:1007D800F230D10001308A004D3082000630831299
:1007E8000313D4009430D3000430D2000030D10079
:1007F80001308A006C30820083120313D301013068
:10080800D4000430D2000D30D10001308A004D30C0
:100818008200063083120313D4009430D3000430CE
:10082800D2001B30D10003308A00533082000311FC
:1008380003191F2C202CB02C831203130510C80198
:1008480064304802031C292C362C83160313AA0192
:10085800FA30A9000000A90B2E2C00008312031304
:10086800C80A242C8312031305144C08DE00043034
:10087800DD004330DC0003308A000230820083123E
:100888000313C90103304902031C4B2C642C831247
:100898000313C80164304802031C532C602C8316D0
:1008A8000313AA01FA30A9000000A90B582C000074
:1008B80083120313C80A4E2C83120313C90A462C49
:1008C800043083120313D4006E30D30003308A003F
:1008D80039308200831203135208CB005108CA0032
:1008E8000310CB1F031403187A2CAF2C83120313A5
:1008F8004A08CC000311CB1B872C0A304A06031D7B
:10090800872C00304B060319962C0311CB1B922C15
:100918000D304A06031D922C00304B06031D952C02
:10092800962CA32C83120313D301D4010430D200D4
:10093800A230D10001308A004D308200AF2C8312E2
:1009480003134A08DD000430DC00AF30DB0001305F
:100958008A00613082001B2C8312031347088A0027
:1009680046088200831603133C08C0003B08013E7A
:100978000318C00A83134018831784000008BD00B9
:1009880083133C1883173B08840000083D060319AD
:10099800CE2CD92C83160313B8010130FF3AB809BD
:1009A800013E0319B80AB700102D83160313C001BE
:1009B80003303D070318C00A3B07BF000318C00AED
:1009C8003C08C0078313401883173F0884000008B9
:1009D800BE00BD0A3C08C0003B08023E0318C00A1E
:1009E800831340188317840000083D020318FD2C68
:1009F800002D83160313BD013C08C0003B08013ECF
:100A08000318C00A83134018831784003D08800028
:100A1800B8013E08B700102D831603133A088A0060
:100A2800390882008313831603133B1883173A0887
:100A380084000008013EBD003B08BF003A08023EA2
:100A48000318BF0A83133F188317840000083D0268
:100A580003182F2D322D83160313BD013B08BF0049
:100A68003A08013E0318BF0A83133F18831784000E
:100A780000083D060319412D482D01308316031344
:100A8800B700B709B70A6A2D8313831603133B18F7
:100A980083173A088400BF010008033E0318BF0A01
:100AA8003A07BE000318BF0A3B08BF0783133F1865
:100AB80083173E0884003C08800083133B18831783
:100AC8003A0884003D088000B7016A2D8316031395
:100AD80039088A0038088200831603130C12380874
:100AE8008A0037088200831203130C081039003A71
:100AF80003090439031D013083160313B700842D3D
:100B08008316031339088A003808820083120313F6
:100B18000C082039003A03090439031D01308316F3
:100B28000313B700972D8316031339088A00380872
:100B38008200053083160313B900A730B8000530CA
:100B48008A008A30820083160313B7080319AD2D73
:100B5800AE2DC12D831203131A0883160313B10097
:100B6800BB012030BA003108BC000530B900C130E3
:100B7800B80005308A001630820083160313300847
:100B88008A002F088200053083160313B900D1307C
:100B9800B80005308A007730820083160313B7083F
:100BA8000319D72DD82D022E83160313BC01333019
:100BB800BB000530BA00E530B90004308A00B63011
:100BC8008200831603133808B2003708B1000310F7
:100BD800B21F03140318F12DF82D831603133108DF
:100BE800831203139900022E063083160313B800EC
:100BF8000230B70005308A00703082008316031374
:100C080030088A002F088200FF00030E83160313A2
:100C180083160313A000A00E0A08A1000408A2006E
:100C28000B1D2B2E260883120313810050308316C8
:100C38000313A707B4300318013EFF3A013EA6008C
:100C48000B11FF30AE1B2B2EAD07031CAE077C0823
:100C5800A3007D08A4007E08A5000630B000393046
:100C6800AF0005308A009D308200063083160313DA
:100C7800B0004330AF0005308A00C73082008316C9
:100C880003132508FE002408FD002308FC002208A1
:100C9800840021088A0020088300FF0E7F0E0900C7
:100CA800643400340A34003410342734E83403340C
:100CB800643400340A3400340034CA349A343B347F
:100CC8000034E134F53405348034963498340034F3
:100CD800403442340F340034A034863401340034B4
:100CE8001034273400340034E8340334003400343A
:100CF80064340034003400340A34003400340034DE
:100D0800303431343234333434343534363437349F
:100D18003834393441344234433444344534463425
:100D2800683465346C346C346F34203477346F3401
:080D380072346C3464340034A1
:02400E00103F61
:00000001FF
